:100000000C9451040C946C040C946C040C946C04CB
:100010000C946C040C946C040C946C040C946C04A0
:100020000C946C040C946C040C946C040C946C0490
:100030000C946C040C946C040C946C040C946C0480
:100040000C946C040C946C040C94F80E0C946C04DA
:100050000C942C070C946C040C94F3060C946C0414
:100060000C9407170C946C040C946C040C946C04A2
:100070000C94A10B0C946C040C946C040D0A0D0AE6
:1000800048573A20466F6C6C6F772D4D65000D0A0E
:10009000466F6C6C6F77204D650A0D536F667477F1
:1000A0006172653A5625642E2564256320000D0A89
:1000B0002D2D2D2D2D2D2D2D2D2D2D2D2D2D2D2D70
:1000C0002D2D2D2D2D2D2D2D2D2D2D2D2D2D000DAD
:1000D0000A005B25695D005B25695D002B20466F8A
:1000E0006C6C6F77204D65202B0048573A20466F87
:1000F0006C6C6F772D4D650053573A2025642E2583
:100100006425630020202020202020202020004E75
:100110006F204750532064617461004C6F6E3A2029
:1001200020202020202020202020202020202000EF
:100130004C61743A202020202020202020202020E4
:100140002020202000416C743A20202020202020F4
:1001500020202020202020202000536174733A2585
:10016000303264204669783A4E6F6E650053617490
:10017000733A25303264204669783A3244202000B0
:10018000536174733A25303264204669783A3344B7
:10019000202000536174733A253032642046697818
:1001A0003A3F3F2020004C6F6E3A20256325642E95
:1001B000252E3364252E336420646567004C6174FA
:1001C0003A20256325642E252E3364252E336420A2
:1001D00064656700416C743A202563253034642ED1
:1001E000252E303364206D004E6F2047505320641D
:1001F000617461005370656564204E3A20202020B0
:100200002020202020202020005370656564204598
:100210003A20202020202020202020202000537061
:1002200065656420543A20202020202020202020B2
:10023000202000536174733A253032642046697877
:100240003A4E6F6E6500536174733A253032642004
:100250004669783A3244202000536174733A25305D
:100260003264204669783A33442020005361747325
:100270003A25303264204669783A3F3F20200053C7
:1002800070656564204E3A20252B346420636D2F01
:100290007300537065656420453A20252B34642033
:1002A000636D2F7300537065656420543A20252BCD
:1002B000346420636D2F73004750532055544320FE
:1002C00054696D650020202020202020202020203F
:1002D0002020202020202020200020204E6F20746D
:1002E000696D652064617461212020202020002038
:1002F00020202020202020202020202020202020FE
:10030000202020002020202020202020202020200D
:10031000202020202020202000446174653A2025E0
:100320003032692F253032692F2530346900546905
:100330006D653A20253032693A253032693A2530E8
:1003400032692E25303369000000211042206330CD
:100350008440A550C660E770088129914AA16BB11D
:100360008CC1ADD1CEE1EFF13112100273325222C5
:10037000B5529442F772D662399318837BB35AA36D
:10038000BDD39CC3FFF3DEE3622443342004011495
:10039000E664C774A44485546AA54BB528850995BD
:1003A000EEE5CFF5ACC58DD5533672261116300665
:1003B000D776F6669556B4465BB77AA7199738870D
:1003C000DFF7FEE79DD7BCC7C448E5588668A77825
:1003D0004008611802282338CCC9EDD98EE9AFF95D
:1003E000488969990AA92BB9F55AD44AB77A966A05
:1003F000711A500A333A122AFDDBDCCBBFFB9EEBAD
:10040000799B588B3BBB1AABA66C877CE44CC55CD4
:10041000222C033C600C411CAEED8FFDECCDCDDDFC
:100420002AAD0BBD688D499D977EB66ED55EF44EA4
:10043000133E322E511E700E9FFFBEEFDDDFFCCF4C
:100440001BBF3AAF599F788F8891A981CAB1EBA1A0
:100450000CD12DC14EF16FE18010A100C230E3201C
:100460000450254046706760B9839893FBA3DAB3C4
:100470003DC31CD37FE35EF3B1029012F322D2326C
:100480003542145277625672EAB5CBA5A895898594
:100490006EF54FE52CD50DC5E234C324A0148104BC
:1004A0006674476424540544DBA7FAB79987B89764
:1004B0005FE77EF71DC73CD7D326F2369106B0160C
:1004C00057667676154634564CD96DC90EF92FE924
:1004D000C899E9898AB9ABA944586548067827685C
:1004E000C018E1088238A3287DCB5CDB3FEB1EFB04
:1004F000F98BD89BBBAB9ABB754A545A376A167AAC
:10050000F10AD01AB32A923A2EFD0FED6CDD4DCDD3
:10051000AABD8BADE89DC98D267C076C645C454CFB
:10052000A23C832CE01CC10C1FEF3EFF5DCF7CDFA3
:100530009BAFBABFD98FF89F176E367E554E745E4B
:10054000932EB23ED10EF01E4572726F722025308E
:1005500032582072656164696E672064617461203D
:1005600066726F6D2073642063617264202852315B
:100570003D25303258292E0D0A000D0A20204D61EC
:100580006E7566616374757265722049443A202500
:10059000690D0A0020204170706C69636174696F95
:1005A0006E2049443A2025730D0A00202050726FB6
:1005B00064756374204E616D653A2025730D0A00E1
:1005C000202050726F64756374205265762E3A2035
:1005D00025692E25690D0A00202053657269616C1A
:1005E000204E6F2E3A200025303258000D0A002090
:1005F000204D616E756661632E20446174653A20FA
:1006000025692F25690D0A0D0A000D0A2053534351
:1006100020696E69742E2E2E006F6B000D0A205318
:10062000444320696E69742E2E2E007265736574C2
:100630002074696D656F75740042616420636D6438
:10064000382052313D253032582E004261642063FB
:100650006D643820523720636865636B2070617465
:100660007465726E2E0D0A004361726420697320F6
:10067000696E636F6D70617469626C6520746F2060
:10068000332E33562E0D0A0042616420636D6435AB
:100690003820523120253032782E004E6F74206180
:1006A0006E2053442D434152442E00436172642016
:1006B000697320696E636F6D70617469626C652027
:1006C000746F20332E33562E004261642041636DD7
:1006D0006434312052313D253032582E00496E6944
:1006E000742074696D656F75742E00496E6974208D
:1006F0006572726F722E004572726F72207365742C
:1007000074696E6720626C6F636B206C656E6774D2
:100710006820746F203531322E004572726F72205E
:1007200072656164696E67204349442E0D0A004575
:1007300072726F722072656164696E672043534400
:100740002E006F6B0D0A000D0A202053442D4341EB
:1007500052442056312E78000D0A202053442D4358
:100760004152442056322E30206F72206C617465E5
:1007700072000D0A20204361706163697479203D25
:10078000202569204D42004E6F204361726420692C
:100790006E20536C6F742E000D0A20534443206466
:1007A00065696E69742E2E2E006F6B004572726F34
:1007B0007220253032582077726974696E67206420
:1007C00061746120746F20736420636172642028F7
:1007D000523D25303258292E0D0A000D0A2046417F
:1007E00054313620696E69742E2E2E0053442D43E9
:1007F00061726420636F756C64206E6F7420626533
:1008000020696E697469616C697A65642E0045724D
:10081000726F722072656164696E6720746865200A
:100820004D42522E004572726F722072656164698A
:100830006E6720746865205642522E005642523A26
:1008400020536563746F722073697A65206E6F74CC
:1008500020737570706F727465642E005642523A40
:1008600020426164206E756D626572206F66207330
:100870006563746F72732E005642523A2050617253
:10088000746974696F6E20697374206E6F7420468A
:100890004154313620747970652E00202E2E2E6F33
:1008A0006B0011241FBECFEFD0E1DEBFCDBF13E040
:1008B000A0E0B1E0EAE7FEE502C005900D92A43C9D
:1008C000B107D9F71DE0A4ECB3E001C01D92A4303C
:1008D000B107E1F70C946E040C940000CFEFD0E167
:1008E000DEBFCDBFF89484B7877F84BF809160005E
:1008F000886180936000109260000E941D13289808
:100900000E94C50E0E946C060E94AD140E94380B16
:100910000E94E7160E94B61778940E94012A289A2E
:1009200029980E94012A8CE790E09F938F931F9251
:100930000E94300C0F900F900F9083E690E09F93F1
:100940008F9381E090E09F938F931F921F928EE888
:1009500090E09F938F931F920E94300C8DB79EB7AB
:1009600009960FB6F8949EBF0FBE8DBF8EEA90E039
:100970009F938F931F920E94300C0F900F900F90B7
:100980008FEC90E09F938F931F920E94300C0E94F7
:10099000650F88EE93E00E94440F9093D1038093FB
:1009A000D0030F900F900F900E94382E0E94C11715
:1009B000882309F425C188EC90E09093E5038093A7
:1009C000E4032091D203822F9927019709F43BC1B8
:1009D00021E02093D203822F99278130910509F4D9
:1009E00017C1029709F438C181E08093D203809146
:1009F000C203882309F4F2C08091650690916606CF
:100A000090937505809374058091630690916406B8
:100A100090937705809376058091590690915A06B8
:100A2000909379058093780580915B0690915C06A0
:100A300090937B0580937A05809161069091620680
:100A400090937D0580937C05809157069091580680
:100A500090937F0580937E0580915D0690915E0660
:100A6000909381058093800580915F069091600648
:100A700090938305809382058091000190910101FC
:100A80009C01220F331F280F391F8091610690911E
:100A90006206002496958795079496958795079406
:100AA000982F802D60E771E00E94EC2E260F371FF3
:100AB00036952795369527953093010120930001AF
:100AC00030938505209384054091CC035091CD034C
:100AD000443651050CF0AFC0253531050CF0B0C0DF
:100AE000E2E0F0E0F093CF03E093CE034F5F5F4F7F
:100AF0005093CD034093CC03F0939505E093940578
:100B000050939705409396056091CA037091CB036B
:100B10006E177F070CF084C0443651050CF480C07A
:100B2000A091E403B091E503109709F079C080919A
:100B3000C8039091C903C3E0893E9C078CF084E60A
:100B400090E09093E5038093E4036F5F7F4F709391
:100B5000CB036093CA03B093C903A093C803CD012C
:100B600065E08C3D96072CF401969093C903809321
:100B7000C803EE0FFF1FE295F295F07FFE27E07F9E
:100B8000FE272E173F0724F02A3431050CF04DC004
:100B9000443651050CF449C080E093E0909308037B
:100BA000809307038091E4039091E503892B31F44E
:100BB00080E797E19093E5038093E4038091C40379
:100BC0009091C50382609093C5038093C4031092F3
:100BD000C20380917A00886C80937A000E94420957
:100BE0000E94D9098091C4039091C503892BB1F06B
:100BF00028980E94382E0E94C117882309F0DBCE66
:100C00002091D203822F99278130910509F0E9CEF6
:100C100029981092C7031092C603E9CE289AC4CE31
:100C20008091C8039091C9039BCF8091C403909198
:100C3000C5038D7FC8CFE091CE03F091CF035CCF89
:100C4000E3E0F0E04FCF8091C4039091C503892B7E
:100C500009F0C1CE22E0BDCE8091D0039091D103A6
:100C60000E944D0F882309F4C2CEC0914B05C130BC
:100C700099F08AEF90E00E94440F9093D103809303
:100C8000D00385B192E0892785B981E090E0909307
:100C9000C7038093C603ABCE88EE93E00E94440F57
:100CA0009093D1038093D0038FEF9FEF90934D05E6
:100CB00080934C05C0934E058CE380934F051092B2
:100CC0005005109251051092520510925305109242
:100CD0005405C093D903D5CFCF93CFB72AE230E0E4
:100CE000F8948091C1008F778093C1008091C100FA
:100CF0008F7B8093C100589A5098599A519A832FAC
:100D000099278093C5002093C4008091C000826021
:100D10008093C00088E18093C1008091C2008F77EA
:100D20008093C2008091C2008F7B8093C20080912B
:100D3000C2008F7D8093C2008091C2008F7E80931D
:100D4000C2008091C200877F8093C2008091C10061
:100D50008B7F8093C1008091C20084608093C20029
:100D60008091C20082608093C2008091C00087FFA2
:100D70000CC08091C6008091C000882334F480911B
:100D8000C6008091C0008823A4F38091C1008068D0
:100D90008093C1008091C10080648093C1008091E4
:100DA0000203909103030E94440F90934B0680939B
:100DB0004A061092D7031092D5031092D4031092D2
:100DC000D30381E08093050310925D0580935E0557
:100DD00082E0809361058AE080935F051092600550
:100DE000CFBFCF9108951F920F920FB60F9211248B
:100DF0008F939F93EF93FF93809105038823A9F42A
:100E00008091DF039091E0030196FC01EC54FA4FCE
:100E1000E081ED3079F08639910561F09093E0033F
:100E20008093DF03E093C6000EC01092E00310929F
:100E3000DF0309C01092E0031092DF0381E080938A
:100E40000503E093C600FF91EF919F918F910F9062
:100E50000FBE0F901F9018951F920F920FB60F9212
:100E600011242F933F934F935F938F939F93AF934F
:100E7000BF93CF93DF93EF93FF935091C600809180
:100E8000D703882309F073C04091E3034423B9F4E6
:100E90005332E1F05D3011F1E42FFF27E755FB4FAE
:100EA00050834F5F4093E3038091E1039091E2030D
:100EB000850F911D9093E2038093E10358C046395A
:100EC00048F38093E3038093D70351C05093A90460
:100ED00081E08093E30383E290E0ECCFA42FBB2773
:100EE000A755BB4FFD01329780812091E1033091DE
:100EF000E203281B3109ED0121978881281B310964
:100F0000C9019F709093E2038093E1030024880F4E
:100F1000991F001C880F991F001C892F902D982F56
:100F2000935C2F733070235C8081891729F01092B5
:100F3000D7031092E3031BC088818217C1F75C932B
:100F40004F5F4093D60381E08093D7038091AB0439
:100F5000823579F788E190E02CE00FB6F894A895F7
:100F6000809360000FBE209360001092E303FF9116
:100F7000EF91DF91CF91BF91AF919F918F915F9151
:100F80004F913F912F910F900FBE0F901F9018958A
:100F9000AC01A0E0B0E09D01A817B90748F4E4EB6C
:100FA000F5E08191280F311D1196A417B507C8F3FC
:100FB0003F70FD01EC54FA4FC9010024880F991FBE
:100FC000001C880F991F001C892F902D835C808343
:100FD0001196FD01EC54FA4F2F733070822F835C11
:100FE0008083AB54BA4F8DE08C93109205038091AF
:100FF000B4058093C6000895BF92CF92DF92EF921E
:10100000FF920F931F93CF93DF93CDB7DEB72C855D
:101010009D857E85BB2483E28093B4059F59909380
:10102000B5052093B60503E010E0772309F4ADC0C1
:10103000CF84D88843E1E42EF12CEC0EFD1EA98963
:10104000BA897150109709F4A0C0109709F43CC0F8
:10105000F601EB0DF11DB3949081119789F477237C
:10106000A1F1F70122E030E0E20EF31ED701C080CB
:10107000D180E20EF31E0D90BC91A02DBB247150C7
:10108000109719F1F601EB0DF11DB3944081119702
:1010900009F466C01097D1F0F601EB0DF11DB39481
:1010A00060811197A1F4772391F0F7013296D7016F
:1010B000CD90DC9032E0E32EF12CEE0EFF1EA081ED
:1010C000B181BB24715003C090E040E060E0F801C2
:1010D000EC54FA4F892F86958695835C80830F5F49
:1010E0001F4FF801EC54FA4F892F992783709070A5
:1010F00082959295907F9827807F982755279A010F
:10110000329522952F7023273F702327822B835CF3
:1011100080830F5F1F4FF801EC54FA4F4F705070EF
:10112000440F551F440F551F862F99270024880F01
:10113000991F001C880F991F001C892F902D842B4C
:10114000835C80830F5F1F4FF801EC54FA4F6F737D
:10115000635C60830F5F1F4F109709F076CF15C057
:10116000772309F4B3CFF701A2E0B0E0EA0EFB1E4B
:10117000D701C080D18022E030E0E20EF31E0D9056
:10118000BC91A02DBB24715085CFC8010E94C80717
:10119000DF91CF911F910F91FF90EF90DF90CF9053
:1011A000BF900895A3E07A2F4091D603465009F4EA
:1011B0005FC0E72FFF27E755FB4F80818D537F5F8F
:1011C000E72FFF27E755FB4F20812D537F5FE72F48
:1011D000FF27E755FB4F30813D537F5FE72FFF2708
:1011E000E755FB4F60816D537F5F9927880F991FEB
:1011F000880F991F522F52955F70582B822F992775
:101200008F70907082959295907F9827807F982715
:10121000232F26952695282B832F9927837090704E
:101220000024969587950794969587950794982F0F
:10123000802D682B41504F3FD9F0EA2FFF27E7550B
:10124000FB4F5083AF5F41504F3F91F0EA2FFF2794
:10125000E755FB4F2083AF5F41504F3F49F0EA2FE6
:10126000FF27E755FB4F6083AF5F442309F0A1CF11
:101270008CEA94E09093D5038093D403A350A09379
:10128000D30308958091D703882309F408950E9419
:10129000D2088091AA048B36E1F18091AB049927A2
:1012A0008736910591F1883691058CF48136910548
:1012B00009F447C08436910509F451C01092D50352
:1012C0001092D4031092D3031092D70308958C3652
:1012D000910549F18D369105FCF48836910571F739
:1012E0008FEF80930403E091D403F091D5038081C4
:1012F0009091EA03892B8093EA03882311F01092DE
:10130000D80381E08093DD03D9CF81E08093DB03B4
:10131000D5CF8091AB04C1CF8637910579F681E0B6
:101320008093DE03CBCF8FEF80930403E091D4034F
:10133000F091D50380818093EB0381E08093DC03FF
:10134000BDCFE091D403F091D503E081E032D8F035
:101350008FE1809306038FEF80930403AFCFE0917A
:10136000D403F091D50390818AE0989FC0011124A5
:101370009093030380930203892B09F49FCF81E0AC
:101380008093DA039BCFE0930603E5CFCF93C82F7A
:101390008A3029F08091C00085FFFCCF04C08DE029
:1013A0000E94C609F7CFC093C60080E090E0CF91BD
:1013B00008951F9380910503882309F457C18091F4
:1013C000DE03882309F066C08091DD03882329F0BD
:1013D00080910503882309F0E1C08091DC03882314
:1013E00029F080910503882309F0ADC02091060300
:1013F0002F3F61F180E190E09F938F93822F992797
:1014000082959295907F9827807F98278E5F9E4F38
:101410009F938F9381E090E09F938F9386E093E07A
:101420009F938F9382E08F938AE08F9381E48F93D1
:101430000E94FC078FEF809306032DB73EB7255F10
:101440003F4F0FB6F8943EBF0FBE2DBF8091DB0318
:10145000882329F080910503882309F059C08091E1
:10146000020390910303892B09F0CBC08091DA032A
:10147000882329F080910503882309F0CCC080914E
:10148000D903882309F4F2C080910503882309F465
:10149000EDC021C080910503882309F495CF8AE02F
:1014A00090E09F938F938DE595E09F938F9381E0DC
:1014B0008F938AE08F9386E58F930E94FC071092AA
:1014C000DE032DB73EB7295F3F4F0FB6F8943EBFFE
:1014D0000FBE2DBF79CF8EE190E09F938F938FE366
:1014E00095E09F938F9381E08F9312E01F9383E7A2
:1014F0008F930E94FC0710934B051092D9038DB770
:101500009EB707960FB6F8949EBF0FBE8DBFAEC0B4
:101510008BE090E09F938F9387E695E09F938F9366
:1015200081E08F938AE08F9387E48F930E94FC077A
:101530001092DB038DB79EB707960FB6F8949EBF47
:101540000FBE8DBF8CCF0E946E0F80E590E09F9301
:101550008F9389E093E09F938F9321E030E03F9356
:101560002F9389E593E09F938F933F932F938BEE77
:1015700093E09F938F9383E08F938AE08F938CE423
:101580008F930E94FC071092DC038DB79EB70F96D5
:101590000FB6F8949EBF0FBE8DBF28CF0E946E0F6E
:1015A00084E190E09F938F939091D80384E1989F7A
:1015B000C0011124875F9C4F9F938F9381E090E03F
:1015C0009F938F9388ED93E09F938F9382E08F9307
:1015D0008AE08F9388E48F930E94FC078091D80360
:1015E0008F5F2DB73EB7255F3F4F0FB6F8943EBFD4
:1015F0000FBE2DBF8430A8F11092D8031092DD03E6
:10160000ECCE80914A0690914B060E944D0F8823A4
:1016100009F030CF2BCF82E490E09F938F9382E745
:1016200095E09F938F9381E08F938AE08F9384E47A
:101630008F930E94FC0780910203909103030E9404
:10164000440F90934B0680934A061092DA032DB70D
:101650003EB7295F3F4F0FB6F8943EBF0FBE2DBF78
:101660000ECF8093D8031092DD03B7CE1F9108955B
:101670004FB72AE230E0F8948091C9008F778093C9
:10168000C9008091C9008F7B8093C9008091C900F7
:101690008F7D8093C9005A9A52985B9A539A832FF0
:1016A00099278093CD002093CC008091C800826060
:1016B0008093C80088E18093C9008091CA008F7729
:1016C0008093CA008091CA008F7B8093CA0080916A
:1016D000CA008F7D8093CA008091CA008F7E80935C
:1016E000CA008091CA00877F8093CA008091C90098
:1016F0008B7F8093C9008091CA0084608093CA0068
:101700008091CA0082608093CA008091C80087FFE0
:101710000CC08091CE008091C800882334F4809161
:10172000CE008091C8008823A4F38091C90080680E
:101730008093C9008091C90080648093C9004FBF25
:1017400008951F920F920FB60F9211242F933F937B
:101750004F935F936F937F938F939F93AF93BF93B9
:10176000EF93FF938091CE000E94B515FF91EF910A
:10177000BF91AF919F918F917F916F915F914F91A9
:101780003F912F910F900FBE0F901F901895982F9B
:1017900080914C06813031F0892F0E94C609282F94
:1017A00033270CC08091E903E82FFF27E75FFC4F48
:1017B00090838F5F8093E90321E030E0C9010895B1
:1017C0000F931F93CF93DF938C01EB01672B71F085
:1017D000F80181918F010E94C70B219739F0F80120
:1017E00081918F010E94C70B219791F7DF91CF91D3
:1017F0001F910F9108950F931F93CF93DF938C0147
:10180000EB01672B81F0F8010F5F1F4F84910E945D
:10181000C70B219741F0F8010F5F1F4F84910E9481
:10182000C70B219781F7DF91CF911F910F910895F9
:10183000CF93C82F181634F480E20E94C70BC15012
:101840001C16D4F3CF910895CF93C82F181634F4F3
:1018500080E30E94C70BC1501C16D4F3CF910895AA
:101860002F923F924F925F926F927F928F929F92B0
:10187000AF92BF92CF92DF92EF92FF920F931F939E
:10188000CF93DF93CDB7DEB7E0970FB6F894DEBF06
:101890000FBECDBF26968FAD26972896EEADFFAD35
:1018A000289788249924540180934C0648E4C42E38
:1018B000D12CCC0EDD1E7F01C701F701149111233D
:1018C00031F0153221F00894E11CF11CF6CFB7017C
:1018D000681B790B09F095C0112309F43DC20894E7
:1018E000E11CF11C1FA63FA4232C0FEF39A6F70122
:1018F0000894E11CF11C14911537C9F1812F806205
:101900008837A9F1103209F440C0133209F48DC0B0
:101910001A3209F479C01D3209F476C01B32C9F1BC
:101920001E32C9F1103309F48AC0812F81538930E6
:1019300008F07EC060E070E0CB01880F991F880F2F
:10194000991F880F991F860F971F680F791F610FC6
:10195000711D60537040F7010894E11CF11C149153
:10196000812F80538A3040F3262E153739F630FE0A
:101970003DC0F60184E090E0C80ED91E80809180C1
:10198000A280B380103209F0C0CF89A5882309F066
:10199000AECF19A7ACCFF7010894E11CF11C14914C
:1019A0001A3209F451C060E070E014C0CB01880F16
:1019B000991F880F991F880F991F860F971F680F0F
:1019C000791F610F711D60537040F7010894E11C8D
:1019D000F11C1491812F80538A3040F3EFEF6F3F59
:1019E0007E0714F46FEF7FEF062F86CFF60182E0BB
:1019F00090E0C80ED91E808191814C01AA24BB249D
:101A000081CF0E94FB0B68CF1A3251F4F60182E0BD
:101A100090E0C80ED91E208022200CF068CF2194BF
:101A200090E1392AEFED3E2262CF98E0392A5FCF6C
:101A30001836C9F01C36D1F481E0382A58CF34FC6E
:101A400056CFF0E23F2A53CFF60182E090E0C80E75
:101A5000D91E608171819FEF6F3F790714F46FEF9A
:101A60007FEF062F44CF24E0322A41CF133609F40A
:101A70004DC1143409F41FC1143609F41CC11936C0
:101A800009F419C11F3409F40FC11F3609F40CC140
:101A9000103709F4F9C0133709F4B2C0153509F449
:101AA000ECC0153709F4E9C0183509F444C01837FB
:101AB00009F441C0112309F44FC1CE0101969DA73D
:101AC0008CA7198381E0482E19A6632C7724042D56
:101AD0005FA4541857FC2DC029A5222331F10F5FB4
:101AE000050DC30180739070892B09F42FC1222347
:101AF00009F027C166FC1BC1C301807390708097F9
:101B000009F410C1852D0E94240C842D992787FD8E
:101B10009095BC018CA59DA50E94E00B64FECCCEE7
:101B2000822D801B0E94180CC7CE66FED9CF0E5F97
:101B3000D7CF5524D1CFE0E1EEA733FE07C0811403
:101B40009104A104B10411F0F0E43F2A19A60FA7F3
:101B500007FD02C02FED3222CE0189969DA78CA7EA
:101B600081149104A104B10419F49FA5992361F192
:101B7000EEA54E2E55246624772418AA84149504C5
:101B8000A604B70410F0F1E0F8ABC501B401A3015D
:101B900092010E94002FDC01CB01082F8A30F0F463
:101BA000005DECA5FDA50293FDA7ECA7C501B4015E
:101BB000A30192010E94002F49015A01F8A9FF23B5
:101BC000E1F62EA5283079F0632C7724CE0101961A
:101BD000482EFCA54F1A28E2420E79CF095A183533
:101BE00001F70F7DDECF632C772463FEEFCF003348
:101BF00069F380E3ECA5FDA58293FDA7ECA7E6CFF2
:101C0000F60182E090E0C80ED91E0190F081E02D2F
:101C1000FDA7ECA7EF2B81F4FE013196FDA7ECA701
:101C200088E289838EE6818385E78B838CE68C83CB
:101C30008D8389E28E831F8207FD15C0802F99272F
:101C400087FD9095AC0160E070E08CA59DA50E9499
:101C5000C02E009731F0482EFCA54F1A04150CF049
:101C600033CF402E31CFECA5FDA501900020E9F740
:101C700031974E2E2CA5421A27CF153511F481E04D
:101C8000382A9AE09EA762CFF60182E090E0C80E63
:101C9000D91E808191814C01AA24BB2490E19EA78A
:101CA000E0E43E2A18E752CF1F3411F4E1E03E2A67
:101CB000F8E0FEA74BCF143411F491E0392A30FE3E
:101CC00018C0F60184E090E0C80ED91E8080918093
:101CD000A280B380B7FE0AC0B094A0949094809480
:101CE000811C911CA11CB11C8DE289A79AE09EA7C2
:101CF0002ECFF60182E090E0C80ED91E808191813E
:101D00004C01AA2497FCA094BA2CE4CFFE01319692
:101D1000FDA7ECA7F60182E090E0C80ED91E8081F5
:101D20008983D0CE822D801B0E94240CEBCE80E3D1
:101D30008AA71BA762E070E0CE018A960E94E00BA2
:101D4000DBCE61E070E0CE018996F8CF822D801B5A
:101D50000E94180C29A5CBCEE0960FB6F894DEBFF2
:101D60000FBECDBFDF91CF911F910F91FF90EF90EC
:101D7000DF90CF90BF90AF909F908F907F906F90AB
:101D80005F904F903F902F9008959FB7F8943F9A9F
:101D9000479884B58C7084BD85B5877385BD85B53E
:101DA000887F826085BD16BC80916E00897F80939C
:101DB0006E0080916E00816080936E0010924E06DE
:101DC00010924D0610924F06109250061092510636
:101DD0001092520610925306109255061092540615
:101DE000109256061092E7031092E6039FBF0895E3
:101DF0001F920F920FB60F9211242F933F938F9340
:101E00009F938091E80381508F3F41F18093E803D5
:101E10008091E4039091E503892BB9F08091E4036C
:101E20009091E50301979093E5038093E4038091FB
:101E3000E4039091E5032091070330910803822386
:101E40009323892B49F4479816C08FEF9FEF909307
:101E5000080380930703F7CF479A0DC089E080936A
:101E6000E8038091E6039091E70301969093E703DE
:101E70008093E603CDCF9F918F913F912F910F904B
:101E80000FBE0F901F9018952091E6033091E70345
:101E9000280F391FC901019708952091E603309159
:101EA000E703821B930B892F990F990B8078089574
:101EB000CF93DF930E94440FEC01CE010E944D0F9F
:101EC0008823D9F3DF91CF91089590E2E9E0F3E020
:101ED0008FE49193815087FFFCCF08959F92AF923A
:101EE000BF92CF92DF92EF92FF920F931F93CF9307
:101EF000DF932091EA0320FF08C08091EB03882341
:101F000009F460C081508093EB0321FF0AC09091D7
:101F1000EB0380915903981709F4F7C19F5F9093E1
:101F2000EB03822F992780FF02C081FD48C00E94E9
:101F3000650F9091EB0380915903891718F48093F2
:101F4000EB03982F9A3088F581E18093E903892F7C
:101F500099279F938F9382ED90E09F938F9381E0D9
:101F60008F930E94300C0F900F900F900F900F9056
:101F70009091EB03E92EFF2481E0E816F10439F19A
:101F800082E0E816F1040CF4C3C182E0E816F10423
:101F900009F453C183E0E816F10409F43BC29150FF
:101FA000909359031092EB033AC380E18093E903C5
:101FB000892F99279F938F9387ED90E0CECF109232
:101FC000EB03B5CF809159038093EB039ECF8091B3
:101FD0001804882309F4DCC18091FB03992782301F
:101FE000910509F458C2833091050CF006C2892B83
:101FF00009F4F7C21092E9038091FA0399279F939D
:102000008F9383E991E09F938F9381E08F930E9458
:10201000300C0F900F900F900F900F90E090EC030A
:10202000F090ED030091EE031091EF0317FDC7C28E
:102030004BE2942EC801B70120E836E948E950E0A8
:102040000E94222F59016A01C801B70120E836E930
:1020500048E950E00E94222FDC01CB01BC01CD01F8
:1020600020E137E240E050E00E94222FE90137FDF5
:10207000A2C2C801B70120E836E948E950E00E9451
:10208000222FDC01CB01BC01CD0120E137E240E091
:1020900050E00E94222FDC01CB01BC01CD012AE0DF
:1020A00030E040E050E00E94222FDA01C90197FDA4
:1020B00094C284E18093E9033F932F93DF93CF93FE
:1020C000BF92AF92892D99279F938F9386EA91E0D3
:1020D0009F938F9381E08F930E94300CE090F003E8
:1020E000F090F1030091F2031091F3038DB79EB7C6
:1020F0000B960FB6F8949EBF0FBE8DBF17FD6AC238
:102100002BE2922EC801B70120E836E948E950E0F9
:102110000E94222F59016A01C801B70120E836E95F
:1021200048E950E00E94222FDC01CB01BC01CD0127
:1021300020E137E240E050E00E94222FE90137FD24
:1021400045C2C801B70120E836E948E950E00E94DD
:10215000222FDC01CB01BC01CD0120E137E240E0C0
:1021600050E00E94222FDC01CB01BC01CD012AE00E
:1021700030E040E050E00E94222FDA01C90197FDD3
:1021800021C288E28093E9033F932F93DF93CF939B
:10219000BF92AF92892D99279F938F938DEB91E0FA
:1021A0009F938F9381E08F930E94300CE090F40313
:1021B000F090F5030091F6031091F7038DB79EB7E9
:1021C0000B960FB6F8949EBF0FBE8DBF17FDF0C1E2
:1021D0008BE2982EC801B70128EE33E040E050E0D2
:1021E0000E94222F59016A01C801B70128EE33E08D
:1021F00040E050E00E94222FDC01CB01EC0197FD72
:10220000D3C18CE38093E903DF93CF93BF92AF9266
:10221000892D99279F938F9384ED91E09F938F93BE
:1022200081E08F930E94300C8DB79EB709960FB650
:10223000F8949EBF0FBE8DBFF2C180911804882311
:1022400009F485C18091FB0399278230910509F437
:10225000D2C1833091050CF411C1039709F4D5C1A3
:102260001092E9038091FA0399279F938F938CE64C
:1022700092E09F938F9381E08F930E94300C0F9098
:102280000F900F900F900F9084E18093E90380915D
:102290000004909101049F938F938FE792E09F93A6
:1022A0008F9311E01F930E94300C88E28093E90322
:1022B0000F900F900F900F900F90809104049091C9
:1022C00005049F938F9382E992E09F938F931F93CE
:1022D0000E94300C8CE38093E9030F900F900F90D5
:1022E0000F900F9080910804909109049F938F9311
:1022F00085EA92E09F938F931F930E94300C0F907A
:102300000F900F900F900F908AC11092EB0309CE9F
:10231000E114F10409F043CE1092E9038CED90E052
:102320009F938F9311E01F930E94300C84E1809360
:10233000E9030F900F900F908AEE90E09F938F9398
:102340001F930E94300C88E28093E9030F900F9056
:102350000F9083E690E09F938F9381E090E09F93AE
:102360008F93FF92EF9288EF90E09F938F931F934C
:102370000E94300C8CE38093E9038DB79EB70996D9
:102380000FB6F8949EBF0FBE8DBF84E091E02CC0C5
:102390008093E9038FE091E09F938F9311E01F9367
:1023A0000E94300C84E18093E9030F900F900F900E
:1023B0008BE191E09F938F931F930E94300C88E2F2
:1023C0008093E9030F900F900F9080E391E09F932B
:1023D0008F931F930E94300C8CE38093E9030F903E
:1023E0000F900F9085E491E09F938F931F930E942D
:1023F000300C0F900F900F9012C1039709F0FACD97
:102400001092E9038091FA0399279F938F9380E8B4
:1024100091E0F9CD1092E90388EB92E09F938F93BE
:10242000C1E0CF930E94300C0F900F900F908091DD
:1024300056068823D1F584E18093E90385EC92E088
:102440009F938F93CF930E94300C88E28093E9038F
:102450000F900F900F908AED92E09F938F93CF9300
:102460000E94300C8CE38093E9030F900F900F9043
:102470008FEE92E09F938F93CF93B9CF892B09F082
:10248000EFCE1092E9038091FA0399279F938F93DF
:1024900083E392E0EECE1092E9038091FA0399274C
:1024A0009F938F938DE691E0AECD84E18093E90315
:1024B00084E093E09F938F93CF930E94300C88E247
:1024C0008093E9030F900F900F9080914D069091AB
:1024D0004E069F938F938091500699279F938F93D9
:1024E00080914F0699279F938F9389E193E09F9363
:1024F0008F93CF930E94300C8CE38093E9038DB7C8
:102500009EB709960FB6F8949EBF0FBE8DBF8091FF
:102510005406909155069F938F9380915306992767
:102520009F938F938091520699279F938F938091C9
:10253000510699279F938F938EE293E09F938F93F9
:10254000CF930E94300C8DB79EB70B9670CE8093C0
:10255000E90388EE91E09F938F9311E01F930E940F
:10256000300C84E18093E9030F900F900F9084EF7B
:1025700091E09F938F931F930E94300C88E2809389
:10258000E9030F900F900F9089E092E09F938F9353
:102590001F930E94300C8CE38093E9030F900F90FF
:1025A0000F908EE192E020CFD095C195DF4F29CEDC
:1025B0009DE2992E0FCED095C195DF4F5ACD5DE2A9
:1025C000952E38CD309521953F4FDBCDD095C195D7
:1025D000DF4FB7CD3DE2932E95CD309521953F4FFE
:1025E00068CD1092E9038091FA0399279F938F9306
:1025F0008AE591E008CD1092E9038091FA039927CA
:102600009F938F9386E492E034CE1092E9038091F9
:10261000FA0399279F938F9389E592E02ACE10922F
:10262000EA03DF91CF911F910F91FF90EF90DF9020
:10263000CF90BF90AF909F900895209A299A219AA9
:10264000289A08959C0160E971E00E94EC2E892B84
:1026500061F0C90183709070892B51F4C90164E65F
:1026600070E00E94EC2E892B19F081E090E0089533
:1026700080E090E008958F929F92AF92BF92CF92A8
:10268000DF92EF92FF920F931F93CF93DF934C0152
:1026900080919104882321F08091680482FD03C019
:1026A000F40111864DC18091680483FFF9CF8091B8
:1026B0005D0490915E04A0915F04B0916004BC0140
:1026C000CD0128EE33E040E050E00E94002F590198
:1026D0006A018091650490916604AA2797FDA095F0
:1026E000BA2F2FE0A216B104C104D10408F01FC113
:1026F0000197A109B10941E75AE369E070E0A40E2E
:10270000B51EC61ED71E7C018D0123E0EE0CFF1CFA
:10271000001F111F2A95D1F7E81AF90A0A0B1B0BA3
:1027200023E837E04BE050E0E20EF31E041F151FD4
:10273000C601B50120E831E541E050E00E94002FDC
:10274000E20EF31E041F151FC801B70121EB3AE387
:1027500042E050E00E94002F80E991E0289FE001D4
:10276000299FD00D389FD00D11242196C801B701A3
:1027700021EB3AE342E050E00E94002F7B018C0104
:102780002CEA3EE840E050E00E94002F84E690E012
:10279000289FB001299F700D389F700D1124C60F1E
:1027A000D71FC801B7012CEA3EE840E050E00E9484
:1027B000002F7B018C0125EB35E040E050E00E94CA
:1027C000002FA901440F551F440F551FC40FD51FDB
:1027D000C801B70125EB35E040E050E00E94002F32
:1027E0007B018C0177E4E71674E0F70670E00707D9
:1027F00070E0170708F098C0C801B7012DE631E076
:1028000040E050E00E94002FA9019E01240F351FD7
:10281000D4012D933C938DE691E0489FE001499FC0
:10282000D00D589FD00D1124CE01AA27BB27E81A3E
:10283000F90A0A0B1B0B0894E11CF11C011D111D68
:10284000C9010E942213882309F46BC04EE853E0AB
:1028500020E0E22FFF27EE0FFF1FEE0FFF1FE40F18
:10286000F51F80819181A281B3818E159F05A007FC
:10287000B10788F484819581A681B7818E159F0563
:10288000A007B10740F02F5FE4012A838081EE2D7D
:10289000E81BEB832CE02F5F2C30D8F2C601B5018A
:1028A00020E831E541E050E00E94002F5B016C011F
:1028B00020E13EE040E050E00E94002FE4012C8344
:1028C000C601B50120E13EE040E050E00E94002F4B
:1028D0005B016C012CE330E040E050E00E94002FEF
:1028E0002D83C601B5012CE330E040E050E00E94AA
:1028F000002F6E8380915D0490915E04A0915F042F
:10290000B0916004BC01CD0128EE33E040E050E01E
:102910000E94002FDC01CB0198878F8381E089879B
:102920000FC04AE553E094CF43E050E06ECFC1EFD3
:10293000DFEFEFEFFFEFAC0EBD1ECE1EDF1EE3CECE
:10294000DF91CF911F910F91FF90EF90DF90CF908B
:10295000BF90AF909F908F90089510929104109225
:102960005C0410923F04109218040895CF93809154
:102970009204909193040E944D0F8823D9F01092F5
:10298000940484E690E00E94440F90939304809313
:10299000920480919404823008F4E5C080919104FF
:1029A000813071F082E08093910480935C04809385
:1029B0003F04D9C0809194048F5F80939404E1CF49
:1029C00080915C04813071F7C0913F04C13051F7B0
:1029D0008091190490911A04019690931A0480939F
:1029E0001904809118048130E9F210921804809142
:1029F00068048093F90380918C048093FA0380919A
:102A000067048093FB038091750490917604A091F4
:102A10007704B09178048093FC039093FD03A09316
:102A2000FE03B093FF038091850490918604A091EA
:102A30008704B09188048093140490931504A093A4
:102A40001604B09317048DE496E00E943B13809126
:102A5000440490914504A0914604B09147048093AA
:102A6000EC039093ED03A093EE03B093EF038091FA
:102A7000480490914904A0914A04B0914B0480937A
:102A8000F0039093F103A093F203B093F3038091CA
:102A9000500490915104A0915204B091530480933A
:102AA000F4039093F503A093F603B093F703C09358
:102AB000F8038091230490912404A0912504B091FF
:102AC00026048093040490930504A0930604B09315
:102AD000070480911F0490912004A0912104B091DB
:102AE00022048093000490930104A0930204B09305
:102AF00003048091270490912804A0912904B091A7
:102B00002A04B095A095909581959F4FAF4FBF4FE8
:102B10008093080490930904A0930A04B0930B04D3
:102B200080912F0490913004A0913104B09132042F
:102B300080930C0490930D04A0930E04B0930F04A3
:102B40008091330490913404A0913504B0913604FF
:102B50008093100490931104A0931204B093130473
:102B6000C09318041FCFCF910895482F209195044A
:102B7000822F99278430910579F18530910594F45D
:102B80008130910509F467C0823091050CF45BC077
:102B90008230910509F48DC0039709F48FC010921B
:102BA0009504DDC08630910509F45AC08630910540
:102BB0003CF18730910509F4A9C0089781F780910D
:102BC0009904481709F4C1C0E0919E04F0919F0454
:102BD000108210929504C3C0842F99279093970474
:102BE0008093960490919804940F90939804809108
:102BF0009904890F8093990485E080939504AFC070
:102C0000842F9927982F8827209196043091970434
:102C1000820F931F90939704809396049091980449
:102C2000940F9093980480919904890F809399044C
:102C3000E0919E04F0919F048081813009F46DC081
:102C4000108286E0DACF892B09F0A9CF453B09F045
:102C5000A6CF81E0D2CF423609F0A1CF82E0CDCF1E
:102C6000E0919A04F0919B0480919C0490919D04C2
:102C7000E817F90708F093CF4193F0939B04E09392
:102C80009A0490919804940F9093980480919904D9
:102C9000890F8093990480919604909197040197ED
:102CA0009093970480939604892B09F058C087E08D
:102CB000A4CF413009F073CF83E09FCF842F9927B1
:102CC00086309105D1F18730910564F5029709F0BE
:102CD00066CF80E494E090939B0480939A044D9691
:102CE00090939D0480939C04019790939F048093FC
:102CF0009E042223A1F184E080939504842F8F5FAA
:102D0000809398048F5F8093990429C080919804E0
:102D1000481709F059CF88E070CF109295040E94AF
:102D2000B6141DC0429709F03ACF8BE194E090931E
:102D30009B0480939A048596D3CF8DE594E090937D
:102D40009B0480939A04C596CBCFE0919E04F091AA
:102D50009F0481E080830E94B614109295048091B4
:102D600000049091010490938705809386058091DB
:102D700004049091050490938905809388058091BF
:102D800008049091090490938B0580938A058091A3
:102D9000FA03992790938D0580938C058091EC031D
:102DA0009091ED0390938F0580938E058091F003B1
:102DB0009091F10390939105809390058091F40395
:102DC0009091F503909393058093920508959FB792
:102DD000F89411B812B88FEF80937E0080917C0038
:102DE0008F7180937C0080917C00807E80937C003A
:102DF00087E080937A0080917B00887F80937B00BE
:102E000080917A00886C80937A009FBF08951F920A
:102E10000F920FB60F9211242F933F938F939F938E
:102E20008091A104282F33278F5F2330310509F4C7
:102E300041C02430310544F52130310509F46CC01E
:102E4000223031050CF44EC08093A10480917800AB
:102E50009091790090935A068093590683E080936D
:102E6000A00480917C00807E9091A004892B8093A7
:102E70007C008091A104882309F46FC080917A00BE
:102E8000886C80937A0069C025303105C9F12530FE
:102E90003105E4F02630310509F44AC02730310508
:102EA00009F452C01092A0041092A10481E0809312
:102EB000C203D7CF8093A1048091780090917900CC
:102EC00090935C0680935B0684E0C9CF8093A10455
:102ED00080917800909179009093620680936106CA
:102EE00085E0BDCF232BF1F68093A104809178007B
:102EF00090917900909366068093650681E0AFCF4C
:102F00008093A10480917800909179009093580665
:102F10008093570686E0A3CF8093A1048091780028
:102F200090917900909364068093630682E097CF36
:102F30008093A104809178009091790090935E062F
:102F400080935D0687E08BCF809178009091790027
:102F50009093600680935F06A5CF9F918F913F91DC
:102F60002F910F900FBE0F901F901895469A3E9884
:102F700082E390E00E94440F9093A3048093A20404
:102F80000895CF93C0E08091A2049091A3040E9481
:102F90004D0F882301F1369B0BC0C093A40482E33C
:102FA00090E00E94440F9093A3048093A20413C066
:102FB0008091A4048F5F8093A404813051F08A3003
:102FC00041F08091A4048A3051F787E08093A404F3
:102FD000E6CFC1E0F6CF8C2F9927CF910895CF92FD
:102FE000DF92EF92FF920F931F93CF93DF938C01A9
:102FF0006A017B0180E090E040E050E060E070E03A
:103000004C155D056E057F05D8F4382F2227E92F72
:10301000FF27D8018D918D019927E827F927EE0F19
:10302000FF1FE85BFC4F80819181822793274F5FD0
:103030005F4F6F4F7F4F4C155D056E057F0528F381
:10304000DF91CF911F910F91FF90EF90DF90CF9084
:1030500008952C9A089584B1806B84B926980E94B3
:10306000291882E58CBD8DB581608DBD2A9A229884
:1030700008950E9429181CBC1DBC08958FEF8EBDB9
:103080000DB407FEFDCF8EB5992708958EBD0DB402
:1030900007FEFDCF08952C980895EF92FF920F93AD
:1030A0001F93CF93DF93EC017A018B0140E0542F03
:1030B000E114F1040105110509F169E0FE01E50FD4
:1030C000F11DE081F7E0440F2E2F33272078307078
:1030D000842F9927807890702817390709F04627A0
:1030E000EE0FF150F7FFEFCF5F5F852F9927AA27EB
:1030F000BB278E159F05A007B10700F3842F9927E2
:10310000880F991F482F4160842F9927DF91CF9115
:103110001F910F91FF90EF9008950F931F93CF93FE
:10312000DF938C010E944B18C8010E94440FEC01F0
:103130000E943E18082FCE010E944D0F882311F4E3
:103140000F3FB1F7802F9927DF91CF911F910F91FA
:103150000895CF92DF92EF92FF920F931F93CF9338
:10316000DF93CDB7DEB726970FB6F894DEBF0FBE5C
:10317000CDBF9A01AB01EE24FF2480648983852FA3
:103180009927AA27BB278A834B833C832D8345E05D
:1031900050E060E070E0CE0101960E944D188E83F1
:1031A0000E9429188FEF0E9446180E944B1884EF46
:1031B00091E00E948D188E010F5F1F4F36E0C32EE5
:1031C000D12CCC0EDD1EF80181918F010E94461892
:1031D0008AE090E00197F1F7C016D106A0F70E94AF
:1031E0003E18282FC7010894E11CF11C855F91400F
:1031F00010F42F3FA1F3822F992726960FB6F8944B
:10320000DEBF0FBECDBFDF91CF911F910F91FF9019
:10321000EF90DF90CF900895EF92FF920F931F935E
:10322000CF93C82F7A018B0140E050E060E070E05E
:1032300087E30E94A91888232CF0B801A7018C2FDE
:103240000E94A9189927CF911F910F91FF90EF909D
:103250000895AF92BF92CF92DF92EF92FF920F93B9
:103260001F93CF93DF935901670178010E94A9183A
:10327000982F8823C9F024E0892F99279F938F9353
:10328000C22FDD27DF93CF9388E495E09F938F9340
:103290001F920E94300C8DB79EB707960FB6F89418
:1032A0009EBF0FBE8DBF26C00E943E18982F807F04
:1032B000F9F09E3FC9F7C0E0D0E0C114D104E104A9
:1032C000F10479F085010E943E18F80181938F0185
:1032D0002196CE01AA27BB278C159D05AE05BF05FB
:1032E00090F30E943E180E943E18C0E0D0E002C059
:1032F0002AE0C2CFCE01DF91CF911F910F91FF90B5
:10330000EF90DF90CF90BF90AF900895AF92BF92B3
:10331000CF92DF92EF92FF920F931F93CF93DF93A1
:10332000CDB7DEB726970FB6F894DEBF0FBECDBF80
:103330006C01DC018C9199279F938F938AE795E02C
:103340009F938F931F920E94300CF601818192818E
:103350009A8389831B820F900F900F900F900F908C
:103360008E010F5F1F4F1F930F9384E995E09F938A
:103370008F931F920E94300C83E090E0C80ED91EFC
:1033800085E0D801F60101900D928A95E1F78DEF65
:103390009FEFC80ED91E1E820F900F900F900F90B6
:1033A0000F901F930F938BEA95E09F938F931F923B
:1033B0000E94300C0F900F900F900F900F90F6011D
:1033C000808599278F7090709F938F9380858295C9
:1033D0008F7099279F938F9380EC95E09F938F93A5
:1033E0001F920E94300C8DB79EB707960FB6F894C7
:1033F0009EBF0FBE8DBF88ED95E09F938F931F9268
:103400000E94300C0F900F900F90F7EEAF2EF5E06A
:10341000BF2EE9E0EE2EF12CEC0CFD1C03E010E0D9
:10342000D7018D917D0199279F938F93BF92AF9282
:103430001F920E94300C0F900F900F900F900F90E2
:103440000150104017FFECCF8CEE95E09F938F93C7
:103450001F920E94300CF6018685482F55274F7029
:10346000507082958F70282F3327858599278295F4
:103470009295907F9827807F9827282B392B20536F
:10348000384F0F900F900F903F932F935F934F9370
:103490008FEE95E09F938F931F920E94300C8DB713
:1034A0009EB707960FB6F8949EBF0FBE8DBF2696A7
:1034B0000FB6F894DEBF0FBECDBFDF91CF911F9145
:1034C0000F91FF90EF90DF90CF90BF90AF90089555
:1034D000EF92FF920F931F93A0E1EA2EF12C012DA2
:1034E000112D9C0140E050E060E070E08AE00E9415
:1034F000291999271F910F91FF90EF900895EF924E
:10350000FF920F931F93B0E1EB2EF12C012D112DA3
:103510009C0140E050E060E070E089E00E942919E1
:1035200099271F910F91FF90EF900895EF92FF92CE
:103530000F931F93CF93DF93CDB7DEB726970FB6C8
:10354000F894DEBF0FBECDBF1A9982C08AE096E024
:103550009F938F931F920E94300C0E942B180F9004
:103560000F900F9089E196E09F938F931F920E9496
:10357000300C0F900F900F908CE196E09F938F93FB
:103580001F920E94300C109267060E9429180F901B
:103590000F900F900EE010E08FEF0E944618015040
:1035A000104017FFF9CF00E010E040E050E060E08D
:1035B00070E080E00E94A918F82E8983C8010F5F8F
:1035C0001F4F855F914008F053C081E0F81669F7FE
:1035D0004AEA51E060E070E088E00E94A91889831F
:1035E00087FD25C182FF4DC081E08093680640E0E1
:1035F00050E060E070E08AE30E94A918898387FDAB
:1036000025C182FDF9C08E010E5F1F4FB5E0EB2E84
:10361000F12CEC0EFD1E0E943E18F80181938F01E3
:10362000EE16FF06C0F78B81992780739070C097C4
:1036300009F448C08BEA96E09F938F931F920E94F3
:10364000300C15E00F900F900F900E942918ADC11B
:103650000E9439181092670611E087E897E09F935F
:103660008F931F920E94300C0F900F900F909DC16E
:103670008BE296E09F938F931F920E94300C12E092
:10368000E1CF82E0809368068E010E5F1F4F85E0D8
:10369000E82EF12CEC0EFD1E0E943E18F8018193DD
:1036A0008F01EE16FF06C0F78D818A3A09F092C0AD
:1036B0008C8199278F709070019709F498CF88E6D4
:1036C00096E0BACF80ED97E00E94440F8C0140E075
:1036D00050E060E070E089E20E940C198983882341
:1036E0000CF493C0C8010E944D0F282F882309F0C5
:1036F00098C0F980F0FCEBCFFF2009F074C040E0E7
:1037000052E060E070E080E10E94A918082F882351
:1037100009F093C08DE696E00E94681A182F88235E
:1037200009F09AC08DE796E00E947F1A182F88232F
:1037300009F0F7C082E497E09F938F931F930E9454
:10374000300C0F900F900F9080917D06829586959A
:10375000869583709927009709F486C0019709F42C
:10376000F3C01092690610926A0610926B061092CE
:103770006C068091680699278130910509F4D9C0BB
:10378000029709F40FC18091690690916A06A09191
:103790006B06B0916C0604E1B695A7959795879551
:1037A0000A95D1F79F938F9382E797E09F938F932A
:1037B0001F920E94300C8DE696E00E94861981E0EF
:1037C000809367060F900F900F900F900F900E94BC
:1037D0002918EBC08BE496E09F938F931F920E9471
:1037E000300C14E02FCF8BEE96E09F938F932F93A6
:1037F0000E94300C13E026CF8BE996E09F938F93C5
:103800001F920E94300C16E01DCF99279F938F9333
:1038100089EC96E09F938F931F920E94300C14E0E6
:10382000D1CF8DED96E09F938F931F92E1CF992793
:103830009F938F9389E396E0EDCF87EF96E09F9378
:103840008F93FF920E94300C1BE0FCCE99279F9330
:103850008F9388E896E0DECF8AE197E09F938F937D
:10386000FF920E94300CEECE309182063F70809124
:103870008306482F5527662777274370507060705E
:103880007070AAE0440F551F661F771FAA95D1F7E5
:10389000809184069927AA27BB27880F991FAA1F02
:1038A000BB1F880F991FAA1FBB1F482B592B6A2BC0
:1038B0007B2B8091850682958695869583709927C6
:1038C000AA27BB27482B592B6A2B7B2B20918606D6
:1038D0002370220F809187069927880F892F881FD0
:1038E000990B9195282B4F5F5F4F6F4F7F4F822F22
:1038F0009927029604C0440F551F661F771F8A95AB
:10390000D2F704C0440F551F661F771F3A95D2F7B0
:103910004093690650936A0660936B0670936C0639
:1039200028CF8FE297E09F938F930F930E94300CE4
:1039300089CE87E497E09F938F931F920E94300C6B
:103940000F900F900F901FCF809184069927AA2780
:10395000BB278F739070A070B070BC0155274427AF
:10396000809185069927AA27BB27BA2FA92F982FC0
:103970008827482B592B6A2B7B2B80918606992709
:10398000AA27BB27482B592B6A2B7B2B83E1440F9B
:10399000551F661F771F8A95D1F740505040684FDA
:1039A0007F4FB6CF88E597E0C6CF812F992726961F
:1039B0000FB6F894DEBF0FBECDBFDF91CF911F9140
:1039C0000F91FF90EF90089588E997E09F938F9370
:1039D0001F920E94300C0E943918109267061092B4
:1039E000690610926A0610926B0610926C0610928D
:1039F00068060F900F900F9089EA97E09F938F933E
:103A00001F920E94300C0F900F900F9080E090E07A
:103A10000895CF92DF92EF92FF920F931F93CF936F
:103A2000DF93DC01CB018A01EE24FF2429E0880F1B
:103A3000991FAA1FBB1F2A95D1F7AC01BD0188E1D0
:103A40000E94A918C82F882309F040C0C3E1D0E024
:103A50000E943E182197D7FFFBCF40E052E060E084
:103A600070E0C8010E94EF176C018EEF0E944618AB
:103A7000E80101501E4F89910E9446180C171D073E
:103A8000D0F78D2D99270E9446188C2D0E9446183C
:103A90000E943E18C82FC7010894E11CF11C855FE5
:103AA0009140A0F52C2F3327C901817190700197A7
:103AB00079F7C9018F7190708B30910569F18C3065
:103AC000910534F50597D9F01CE001C014E08C2F66
:103AD00099279F938F93C12FDD27DF93CF938CEA94
:103AE00097E09F938F931F920E94300C8DB79EB7E3
:103AF00007960FB6F8949EBF0FBE8DBF27C080ED0E
:103B000097E00E948D18C82F8F3F41F017E0DFCF5C
:103B10004D97D1F619E0DBCF18E0D9CF40E050E067
:103B200060E070E08DE00E94A918C82F882341F45E
:103B30000E943E18C82F882339F4C0E0D0E006C0A8
:103B400014E00E943E18C3CF19E0FBCFCE01DF91F5
:103B5000CF911F910F91FF90EF90DF90CF9008953C
:103B6000EF92FF920F931F93DC01CB019A0159E072
:103B7000880F991FAA1FBB1F5A95D1F7E12C42E06D
:103B8000F42E012D112DAC01BD0181E10E942919F6
:103B900099271F910F91FF90EF900895FC01892BB9
:103BA00019F08185882329F420E030E040E050E0DE
:103BB00063C0808191818C5B97409C01442755278D
:103BC000A9E1220F331F441F551FAA95D1F7828107
:103BD0009927AA27BB278F709070A070B07075E1ED
:103BE000880F991FAA1FBB1F7A95D1F7282B392B55
:103BF0004A2B5B2B83819927AA27BB278F71907053
:103C0000A070B070DC0199278827282B392B4A2B0C
:103C10005B2B84819927AA27BB278F719070A07096
:103C2000B0707BE0880F991FAA1FBB1F7A95D1F750
:103C3000282B392B4A2B5B2B85819927AA27BB2759
:103C40008F739070A070B07065E0880F991FAA1FE5
:103C5000BB1F6A95D1F7282B392B4A2B5B2B86810A
:103C600086959927AA27BB278F719070A070B07096
:103C7000282B392B4A2B5B2BCA01B9010895A0E0F0
:103C8000B0E060E0AD019A012C55394FF901E15ED9
:103C9000FD4F8081882331F06F5F405E5D4F633060
:103CA00090F303C0D90181E08083CD01089500978E
:103CB00071F020E0E4EAF6E0E817F90749F02F5F39
:103CC000E05EFD4F2330C0F380E090E0089508955A
:103CD000E15EFD4F1082EF51F2401082118212829C
:103CE000138214821582168217821086128611861C
:103CF00013861486158616861786108A118A128AEC
:103D0000138AE55EFD4F1082118212821382EB51FD
:103D1000F240148A158A168A178A118E108E128E16
:103D200081E090E00895CF93DF93DC01EB0140E068
:103D300050E030E08C918F3239F442C08F3251F034
:103D40003F5F4115510559F4FD01E30FF11D8081DD
:103D50008823A1F7AF013F5F41155105A9F31B86E9
:103D600080E2FE012AE08193215027FFFCCF30E062
:103D7000232F8C918F3279F1E32FFF27CF018A0F08
:103D80009B1F84179507D0F42B3038F5EA0FFB1FE3
:103D900090819E32D9F0892F81568A3198F4FE01A4
:103DA000E20FF11D905290833F5F2F5FE32FFF27BB
:103DB000CF018A0F9B1F8417950730F3CA010FC0EC
:103DC00031E0C2CFFE01E20FF11DEDCF293028F422
:103DD0003F5F28E0D1CF31E0CFCF80E090E0DF91AE
:103DE000CF9108959C0180918D06882329F420E0CD
:103DF00030E040E050E021C02230310510F422E0F4
:103E000030E02250304080918E069927289FA001F3
:103E1000299F500D389F500D1124CA019C01442741
:103E2000552780919C0690919D06A0919E06B09189
:103E30009F06280F391F4A1F5B1FCA01B901089549
:103E4000CF93DF93FC01EB0180918D06882319F459
:103E500080E090E019C080919C0690919D06A09111
:103E60009E06B0919F06C81BD90BEA0BFB0B8091F5
:103E70008E06282F332744275527BE01CF010E94E5
:103E8000002FDA01C9010296DF91CF910895809148
:103E90008D06992708955F926F927F928F929F92DD
:103EA000AF92BF92CF92DF92EF92FF920F931F9348
:103EB000CF93DF93CDB7DEB7C050D2400FB6F894A2
:103EC000DEBF0FBECDBF9C016624772443018091E5
:103ED0008D06882309F47FC044275527220F331FFE
:103EE000441F551FDA01C90169E0B695A79597955A
:103EF00087956A95D1F7E0909406F0909506009129
:103F0000960610919706E80EF91E0A1F1B1F9FEFD9
:103F1000A92E91E0B92EC12CD12CA222B322C42209
:103F2000D5223BC081E0582E1182108244275527AC
:103F3000220F331F441F551FDA01C90119E0B6953E
:103F4000A795979587951A95D1F7E0909406F090EC
:103F500095060091960610919706E80EF91E0A1F25
:103F60001B1FBEEFAB2EB1E0BB2EC12CD12CA22269
:103F7000B322C422D522E614F7040805190511F46A
:103F8000552049F4AE014F5F5F4FC401B3010E9459
:103F9000091D882301F5552009F1E614F7040805E9
:103FA000190559F037014801AE014F5F5F4FC80155
:103FB000B7010E94B01D882371F4FE013196EA0D0D
:103FC000FB1D20813181C90102978E5E9F4F08F44D
:103FD000A9CF5524A9CF80E090E002C081E090E015
:103FE000C050DE4F0FB6F894DEBF0FBECDBFDF91DD
:103FF000CF911F910F91FF90EF90DF90CF90BF90E6
:10400000AF909F908F907F906F905F900895CF9228
:10401000DF92EF92FF920F931F93CF93DF93EC0108
:10402000892B09F474C080918D06882309F46FC030
:104030008B8599278136910521F08737910509F005
:1040400066C089859A85892B09F049C0ABE1EA2EC3
:10405000F12CEC0EFD1EFBE1CF2EF2E0DF2ECC0E9C
:10406000DD1E8C899D89AE89BF89F601808391838D
:10407000A283B383A701BC01CD010E94B01D882398
:1040800009F043C0088D198D000F111F029512957C
:10409000107F1027007F10270E0D1F1D8C859D851A
:1040A000AE85BF85F801848F958FA68FB78F8DE47D
:1040B00096E00E94CE1DDC01CB01F801868B978B28
:1040C000A08FB18FA701F6016081718182819381F8
:1040D0000E94091D8823C9F480E090E01AC01BE10A
:1040E000E12EF12CEC0EFD1EBBE1CB2EB2E0DB2E5F
:1040F000CC0EDD1EA701F601608171818281938162
:104100000E94091D882309F4ACCF0E94A7208FEFDD
:104110009FEFDF91CF911F910F91FF90EF90DF9074
:10412000CF9008950F931F93CF93DF93EC010FEF80
:104130001FEF009731F00E9407208C01CE010E94F2
:10414000571EC801DF91CF911F910F910895EF92F3
:10415000FF921F93CF93DF93EE24FF24C4EAD6E0AF
:1041600012E0C15EDD4F8881CF51D240813031F005
:104170001150C05EDD4F17FFF4CF06C0CE010E9484
:104180009220E80EF91EF4CF0E94E41C10928D06D6
:104190008E2D9927DF91CF911F91FF90EF90089579
:1041A0002F923F924F925F926F927F928F929F9247
:1041B000AF92BF92CF92DF92EF92FF920F931F9335
:1041C000CF93DF93CDB7DEB724970FB6F894DEBF59
:1041D0000FBECDBFAC011A82198280918D06882353
:1041E00009F488C04115510509F484C08824992434
:1041F00054019BE1292E92E0392E240E351E8A01AE
:10420000055E1F4F2401350180919406909195061B
:10421000A0919606B0919706880D991DAA1DBB1D09
:10422000F10180839183A283B383A801BC01CD01F6
:104230000E94B01D882309F05BC01C821B827301A1
:104240006201F694E794D794C79409C0AB81BC810E
:104250001196BC83AB83AF3FB10509F058F5EB81F4
:10426000FC81EE0FFF1FE00FF11F80819181892BF0
:1042700069F78FEF9FEF91838083A801D1016D9142
:104280007D918D919C910E94091D882389F5EB8178
:10429000FC81EC0DFD1DFA83E98380E091E09C83B5
:1042A0008B83AB81BC811196BC83AB83AF3FB105DF
:1042B000B1F2A8F20894811C911CA11CB11C80E0F1
:1042C00092E0A0E0B0E0480E591E6A1E7B1E80916D
:1042D000920690919306AA27BB2788169906AA06EC
:1042E000BB0640F4A981BA81AB2B09F48DCF02C083
:1042F0000E94A72089819A8124960FB6F894DEBF88
:104300000FBECDBFDF91CF911F910F91FF90EF9026
:10431000DF90CF90BF90AF909F908F907F906F90E5
:104320005F904F903F902F900895AF92BF92CF92A1
:10433000DF92EF92FF920F931F93CF93DF938C0145
:10434000EE24FF2480918D06882309F489C001158D
:10435000110509F485C080919C0690919D06A0915D
:104360009E06B0919F06F8012481358146815781D0
:10437000281739074A075B0708F472C08091A00626
:104380009091A106A091A206B091A306821793076F
:10439000A407B50708F464C0CA01B9010E94201F30
:1043A0007C01C701AA27BB27880F991FAA1FBB1F23
:1043B0009C01AD0169E056954795379527956A951B
:1043C000D1F7C0919406D0919506E0919606F091B0
:1043D0009706C20FD31FE41FF51F2FEFA22E21E077
:1043E000B22EC12CD12CA822B922CA22DB229801DC
:1043F000255E3D4FD9014D915D916D917C91139753
:104400004C175D076E077F0771F0CD93DD93ED9339
:10441000FC931397C8014B96AC01BE01CF010E94DB
:10442000B01D882369F4F801EA0DFB1DE38CF48CC0
:10443000B8EFEB16BFEFFB0630F0EE24FF2410C000
:104440000E94A7200DC0C7010E94F21EDC01CB0113
:10445000F80184839583A683B7831086128611861C
:10446000C701DF91CF911F910F91FF90EF90DF90E7
:10447000CF90BF90AF9008952F923F924F925F924E
:104480006F927F928F929F92AF92BF92CF92DF9264
:10449000EF92FF920F931F93CF93DF93CDB7DEB7C9
:1044A0002E970FB6F894DEBF0FBECDBF9A838983D7
:1044B0006B834C8319011A86198600E080918D0662
:1044C000882309F4B0C0232B09F4ADC029813A81B7
:1044D000232B09F4A8C0D1011D921D921D921C929C
:1044E0001397F101C488D588E688F788C114D104F0
:1044F000E104F10409F09AC0809190069091910630
:10450000880F991F82959295907F9827807F982792
:10451000892F992786959C01442755272D833E8313
:104520004F8358878091980690919906A0919A069A
:10453000B0919B0680839183A283B383F101808134
:104540009181A281B3810097A105B10509F40FC142
:104550009101255E3D4F3C872B871BE1812E912CDD
:10456000820C931C9C01AD01F10184839583A68389
:10457000B7831086128611864424552432015901CE
:104580006A01A40CB51CC61CD71CAB85BC85AD92BA
:10459000BD92CD92DC921397A401C601B5010E9491
:1045A000B01D8823F1F5EE24FF24A701440F551F09
:1045B00042955295507F5427407F5427FA01E80DC9
:1045C000F91DFE87ED872081822F9927009751F0F2
:1045D000853E910539F08385FC818F233B818317CC
:1045E00009F457C00894E11CF11CF0E1EF16F10446
:1045F000E0F20894411C511C611C711C2D813E810C
:104600004F815885421653066406750608F0E7C0C8
:10461000002309F0E4C0F1012481358146815781EE
:10462000AECF0E94A72080E090E00FC18091980655
:1046300090919906A0919A06B0919B06C816D9064A
:10464000EA06FB0608F470C080919C0690919D06D6
:10465000A0919E06B0919F06C816D906EA06FB06F1
:1046600008F06AC08091900690919106880F991F7A
:1046700082959295907F9827807F9827892F9927F8
:1046800086959C01442755272D833E834F83588769
:1046900055CF30E0A981BA818C91281709F0A2CFBB
:1046A0003F5F3B3078F4632F7727AD85BE85A60F3B
:1046B000B71FE981FA816E0F7F1F9C91DB018C91FE
:1046C000981771F33A3008F48DCF8A01080D191D3F
:1046D000F8018385F101828FF801828D938D0E940C
:1046E000F21EDC01CB01F10180839183A283B383AD
:1046F00084839583A683B783108612861186A48A45
:10470000B58AC68AD78AF18EE08EF801848D958DA0
:10471000A68DB78DF10184879587A687B78701E0BD
:10472000E0E1EE2EF12C5ECF80919C0690919D06EB
:10473000A0919E06B0919F06C816D906EA06FB0610
:1047400008F471CF8091A0069091A106A091A206D5
:10475000B091A3068C159D05AE05BF0508F463CF87
:1047600080918E06282F3327442755278DCF91011E
:10477000255E3D4F3C872B87D901CD92DD92ED928E
:10478000FC9213979BE1892E912C820C931CA4011F
:10479000C701B6010E94B01D882309F042CFF10184
:1047A000A08DB18DAA0FBB1FA295B295B07FBA277D
:1047B000A07FBA27A80DB91D8C919927009709F4FD
:1047C00032CF853E910509F42ECFFD0183859927CF
:1047D0009C012071307084FD2BC0C90136C00023BC
:1047E00091F480919C0690919D06A0919E06B091B7
:1047F0009F06F101248135814681578128173907A9
:104800004A075B0760F429853A85232B71F0002362
:1048100061F4F1012481358146815781ADCEC1011A
:104820000E9495219A878987EECF802F99270DC006
:10483000FD01828D938D0E94F21EDC01CB01F101FE
:1048400080839183A283B3838DCE2E960FB6F89486
:10485000DEBF0FBECDBFDF91CF911F910F91FF90B3
:10486000EF90DF90CF90BF90AF909F908F907F9010
:104870006F905F904F903F902F900895BF92CF928E
:10488000DF92EF92FF920F931F93CF93DF93CDB7F9
:10489000DEB72C970FB6F894DEBF0FBECDBFFC017C
:1048A000B62EC42E790100E010E0DD24892B39F00A
:1048B0002115310521F080918D06882319F480E0BF
:1048C00090E033C0DF01F901148A158A168A178A2D
:1048D000118F008F8C918823C1F48D2D992725C0CD
:1048E0006B2D4C2D9701CE0101960E943C2288230E
:1048F000A1F3F8018081882311F461E0D62ED8015C
:104900008C91882351F3DD2041F7BE016F5F7F4F0B
:10491000CD010E94931E8C010097F9F2FC01808169
:104920008823F1F260E148E1DDCF2C960FB6F894D0
:10493000DEBF0FBECDBFDF91CF911F910F91FF90D2
:10494000EF90DF90CF90BF900895AF92BF92CF923B
:10495000DF92EF92FF920F931F93CF93DF93EC01BF
:10496000EE24FF248701E1E0CE2ED12C80918D062C
:10497000882309F45DC0209709F45AC02115310538
:1049800041F02230310509F465C0E888F9880A89C8
:104990001B89E40EF51E061F171F17FD4CC08C85E2
:1049A0009D85AE85BF858E159F05A007B1070CF4C8
:1049B00042C088819981AA81BB818C839D83AE830B
:1049C000BF8318861A861986188A198A1A8A1B8A3A
:1049D00080E090E0A0E0B0E08E159F05A007B10751
:1049E00070F5A12C72E0B72E12C01A861986888540
:1049F0008F5F888790918E06891788F588899989B5
:104A0000AA89BB898E159F05A007B107C0F401963E
:104A1000A11DB11D888B998BAA8BBB8B89859A852B
:104A2000019622E08030920700F79A878987E6CFC7
:104A300080E090E021C088899989AA89BB898E1578
:104A40009F05A007B10711F0C60116C0CC24DD24D4
:104A5000C60112C0EC84FD840E851F859ACFCE015D
:104A60000E949521892B11F01886C8CF8885815026
:104A70008887BA86A986C2CFDF91CF911F910F9107
:104A8000FF90EF90DF90CF90BF90AF9008956F921E
:104A90007F928F929F92AF92BF92CF92DF92EF92CE
:104AA000FF920F931F93CF93DF938C01EE24FF248B
:104AB00080918D06882349F00115110531F0C80158
:104AC0000E94D0207C01892B11F4C7017FC022E015
:104AD00030E040E050E060E070E0C8010E94A524B2
:104AE000F80164817581868197810E94201FAA2721
:104AF000BB27880F991FAA1FBB1F9C01AD0169E04E
:104B000056954795379527956A95D1F7C0919406A4
:104B1000D0919506E0919606F0919706C20FD31FAB
:104B2000E41FF51F2FEF622E21E0722E812C912CB5
:104B3000682279228A229B22BBE1AB2EB2E0BB2EF7
:104B4000A00EB11ED5012D913D914D915C91139711
:104B50002C173D074E075F0779F1CD93DD93ED9359
:104B6000FC931397ABE1CA2ED12CC00ED11EA60127
:104B7000BE01CF010E94B01D882321F5F801E60D8A
:104B8000F71DF48EE38EA601F501608171818281AB
:104B900093810E94091DC82F8823A1F4C7010E9498
:104BA000F21EDC01CB01F80184839583A683B783D1
:104BB000C0871286118689CFFBE1CF2ED12CC00E83
:104BC000D11EDCCF0E94A72080E090E0DF91CF9142
:104BD0001F910F91FF90EF90DF90CF90BF90AF901B
:104BE0009F908F907F906F9008959F92AF92BF9209
:104BF000CF92DF92EF92FF920F931F93CF93DF93A9
:104C0000EC01A1E09A2E80918D06882309F452C010
:104C1000209709F44FC0EE24FF248701FE01EE0D1A
:104C2000FF1D138E0894E11CF11C011D111D80E075
:104C3000E81682E0F80680E0080780E0180770F3C5
:104C4000EE24FF24870180918E068823B1F1FBE1D9
:104C5000AF2EF2E0BF2EAC0EBD1EEBE1CE2ED12C5E
:104C6000CC0EDD1E0FC00894E11CF11C011D111DAE
:104C700080918E069927AA27BB27E816F9060A070E
:104C80001B07D8F48C819D81AE81BF818E0D9F1D45
:104C9000A01FB11FF50180839183A283B383A60176
:104CA000BC01CD010E94091D8823E9F20E94A720C2
:104CB0009924D9CF80E090E002C0892D9927DF9117
:104CC000CF911F910F91FF90EF90DF90CF90BF9009
:104CD000AF909F9008952F923F924F925F926F9264
:104CE0007F928F929F92AF92BF92CF92DF92EF927C
:104CF000FF920F931F93CF93DF93CDB7DEB76197EA
:104D00000FB6F894DEBF0FBECDBF9A838983362ECF
:104D10008A01CC24DD24DC86CB86DE86CD86222467
:104D200080918D06882309F480C04115510509F44E
:104D30007CC029813A81232B09F477C0DA011D92C6
:104D40001D921D921C921397FA01A488B588C688FB
:104D5000D788A114B104C104D10409F069C08091BD
:104D6000900690919106880F991F82959295907F59
:104D70009827807F9827892F992786959C0144271B
:104D800055272F83388749875A874D855E855C87ED
:104D90004B878091980690919906A0919A06B091C0
:104DA0009B0680839183A283B383F80180819181E4
:104DB000A281B3810097A105B10509F07BC0055E12
:104DC0001D4FD801AD92BD92CD92DC9213970B513D
:104DD0001240FBE1EF2EF12CE00EF11EA701C601FF
:104DE000B5010E94B01D8823F1F4F801A08DB18DAA
:104DF000AA0FBB1FA295B295B07FBA27A07FBA2792
:104E0000AE0DBF1D8C919927009779F0853E9105D5
:104E100061F0FD01838599279C012071307084FD2C
:104E20003AC0C901B1C10E94A72080E090E0ACC1A6
:104E30008091980690919906A0919A06B0919B0650
:104E4000A816B906CA06DB0608F454C180919C0670
:104E500090919D06A0919E06B0919F06A816B90656
:104E6000CA06DB0608F04EC180919006909191062B
:104E7000880F991F82959295907F9827807F982719
:104E8000892F992786959C01442755272F8338879A
:104E900049875A878ACFFD01A28DB38DBC87AB8726
:104EA000CD010E94F21EDC01CB01F80180839183C9
:104EB000A283B383C8010E94D0203C01892B09F44E
:104EC00016C1D8012D913D914D915C91F80124833B
:104ED00035834683578310867BE1472E72E0572E39
:104EE000400E511E6BE1E62EF12CE00EF11E1B82EE
:104EF0001C821D821E828B809C80AD80BE80820EB3
:104F0000931EA41EB51ED2018D929D92AD92BC92AD
:104F10001397A701C501B4010E94B01D882309F0B1
:104F200082CFCC24DD240AC0853EB1F00894C11C98
:104F3000D11CB0E1CB16D10408F068C0F601EE0F29
:104F4000FF1FE295F295F07FFE27E07FFE27EE0D32
:104F5000FF1D8081882341F7F98BE88BDF012981D0
:104F60003A819AE0F90181919F018D93915097FFC9
:104F7000F9CFE889F9893386738E628E8DE496E0E5
:104F80000E94CE1DDC01CB01E889F989868B978BC5
:104F9000A08FB18F148E158E168E178EA701D20199
:104FA0006D917D918D919C910E94091D8F87882321
:104FB00009F09BC0C3010E94F21EDC01CB01F80185
:104FC00080839183A283B38384839583A683B783ED
:104FD0002F85208712861186328E148615861686B6
:104FE0001786848A958AA68AB78AD18EC08E34FCA9
:104FF0002CC081E0282EB0E1CB2ED12C0894C11C0E
:10500000D11CB0E1CB16D10408F498CF2B813C81A0
:105010004D815E812F5F3F4F4F4F5F4F2B833C830E
:105020004D835E838F819885A985BA8528173907B6
:105030004A075B0708F081C0222009F07EC0F80112
:10504000248135814681578156CFC8010E94F525BC
:10505000F80180819181A281B381F20180839183E3
:10506000A283B383A701BC01CD010E94B01D882398
:10507000E1F52EE2F801238F20E2F701319699E065
:105080002193915097FFFCCF80E1F7018387738EC6
:10509000628E168A178A108E118E148E158E168EB9
:1050A000178E3EE230A331A3822FB29698E081930F
:1050B000915097FFFCCF80E1F70183A72B853C85BA
:1050C00033AF22AF16AA17AA10AE11AE14AE15AEAA
:1050D00016AE17AEA701D2016D917D918D919C9175
:1050E0000E94091D882309F484CF0E94A720822DE5
:1050F00099274AC080919C0690919D06A0919E069A
:10510000B0919F06A816B906CA06DB0608F48DCE34
:105110008091A0069091A106A091A206B091A3064D
:105120008A159B05AC05BD0508F47FCE80918E06DF
:10513000282F332744275527A9CE2220B9F4809160
:105140009C0690919D06A0919E06B0919F06F80145
:105150002481358146815781281739074A075B0723
:1051600028F0C8010E9495219E878D872D853E8558
:10517000232B09F4BCCF222009F0B9CFF8012481F8
:10518000358146815781B3CE61960FB6F894DEBF64
:105190000FBECDBFDF91CF911F910F91FF90EF9088
:1051A000DF90CF90BF90AF909F908F907F906F9047
:1051B0005F904F903F902F900895BF92CF92DF92D3
:1051C000EF92FF920F931F93CF93DF93CDB7DEB78C
:1051D0002C970FB6F894DEBF0FBECDBF9C01B62E44
:1051E0007A0100E010E0CC24892B39F041155105FB
:1051F00021F080918D06882319F480E090E041C071
:10520000D901FA01148A158A168A178A118F008F1C
:105210008C91882331F58C2D992733C0D62E970198
:1052200048E16D2DCE0101960E943C22882399F41D
:10523000F8018081882309F4DB2CA7016D2DCE01B4
:1052400001960E946B26882331F3F8018081882320
:1052500011F441E0C42ED8018C918823E1F2CC20D6
:10526000D1F6BE016F5F7F4FCD010E94931E8C016E
:10527000009789F2FC016081662381F250E1D52E0E
:10528000CECF2C960FB6F894DEBF0FBECDBFDF9108
:10529000CF911F910F91FF90EF90DF90CF90BF9033
:1052A0000895FF920F931F93CF93DF938C01F62EF7
:1052B000C0E0D0E080918D06882309F49BC00115E1
:1052C000110509F497C00E943F1EEC01892B09F4D7
:1052D00091C0188219821A821B821C821D821E8232
:1052E0001F8218861A861986FB861C861D861E86D6
:1052F0001F86188A198A1A8A1B8AC55EDD4F188292
:1053000019821A821B82CB51D2401C8A1D8A1E8AA6
:105310001F8A198E188E1A8E9E0148E16885C80171
:105320000E943E24882309F441C06F2D772767FD32
:1053300070956237710509F45AC0633771050CF432
:1053400045C067377105E1F58A8D99278C01017099
:10535000107080FD35C0688179818A819B810E94AF
:10536000201F0E944B1FCE010E94D0200E94F21EDF
:10537000DC01CB0188839983AA83BB838C839D83C3
:10538000AE83BF8318861A8709871C861D861E86F2
:105390001F86188A198A1A8A1B8A980140E050E0F1
:1053A00060E070E0CE010E94A52424C06F2D772715
:1053B00067FD70956136710591F06737710579F079
:1053C000CE010E949220C0E0D0E014C06136710589
:1053D000B9F78A8D80FDF4CF22E030E0DFCFAE0157
:1053E00060E2C8010E94DD28882321F4E9CF20E093
:1053F00030E0D4CFCE01DF91CF911F910F91FF907C
:1054000008958F929F92AF92BF92CF92DF92EF92C8
:10541000FF920F931F93CF93C0E08BED97E09F9384
:105420008F93CF930E94300CC0938D060F900F90F6
:105430000F90E3ECF8E082E01082E05EFD4F8150D7
:1054400087FFFACF0E94961AC82F882309F0A9C0B7
:105450004FEB56E060E070E080E090E00E94B01D0D
:10546000882309F0EAC080918108843009F4C2C021
:10547000863009F4BFC08E3009F4BCC0882499245A
:1054800054018091CA069091CB068050924009F059
:10549000CBC08091CC0680938E064091CF0640937E
:1054A0008F06C090D006D090D106D0929106C092BF
:1054B00090062091D5063091D6063093930620931E
:1054C00092068091CD069091CE067C01002711278F
:1054D000E80CF91C0A1D1B1DE0929406F09295063B
:1054E0000093960610939706C901AA27BB27242F7D
:1054F000332744275527BC01CD010E94CD2EDC0166
:10550000CB018E0D9F1DA01FB11F80939806909315
:105510009906A0939A06B0939B06D294C2946FE02A
:10552000C622CD24D622CD24960144275527280F04
:10553000391F4A1F5B1F20939C0630939D064093A2
:105540009E0650939F068091DF069091E006A09101
:10555000E106B091E2060097A105B10509F476C015
:10556000280F391F4A1F5B1F2150304040405040D8
:105570002093A0063093A1064093A2065093A30661
:105580008091F506863421F48091F6068134B9F0D5
:1055900088E798E09F938F931F920E94300CC6E09B
:1055A00008C08CEE97E09F938F931F920E94300C5F
:1055B000C1E00F900F900F900E94A72050C08091E3
:1055C000F706843529F78091F806813309F7809131
:1055D000F9068633E9F681E080938D06C0E08BE919
:1055E00098E09F938F93CF930E94300C0F900F9071
:1055F0000F9035C08090850890908608A09087080D
:10560000B09088084FEB56E0C501B4010E94B01D70
:10561000882309F436CF85E298E09F938F931F92F9
:105620000E94300CC3E0C5CF8CE398E09F938F932A
:105630001F920E94300CC4E0BCCF8EE098E09F9394
:105640008F93CF930E94300CC2E0B3CF8CE598E0EB
:105650009F938F931F920E94300CC5E0AACF8C2F8E
:105660009927CF911F910F91FF90EF90DF90CF90EE
:10567000BF90AF909F908F900895AF92BF92CF92BE
:10568000DF92EF92FF920F931F93CF93DF93EC0182
:105690007FEFA72EB72E80918D06882309F472C064
:1056A000209709F46FC02C853D854E855F852115B7
:1056B00031054105510509F465C0C888D988EA88D3
:1056C000FB88D701C6010196A11DB11D8217930762
:1056D000A407B50708F056C00C811D812E813F81BB
:1056E0008885080F111D211D311DFE01E55EFD4F4E
:1056F00080819181A281B38180179107A207B307AE
:1057000089F00083118322833383CE014B96AC0151
:10571000C901B8010E94B01D882351F5C888D988F5
:10572000EA88FB8889859A85FE01E80FF91F238D99
:10573000A22EBB240894C11CD11CE11CF11CC88AF8
:10574000D98AEA8AFB8A019622E080309207C0F06B
:105750001A86198688858F5F888790918E068917AB
:1057600088F0CE010E949521892B29F018860AC065
:105770000E94A72007C088858150888780E092E03A
:105780009A878987C501DF91CF911F910F91FF9073
:10579000EF90DF90CF90BF90AF9008958F929F923F
:1057A000AF92BF92DF92EF92FF920F931F93CF932E
:1057B000DF93D82E8B0180918D06882309F46FC06A
:1057C0006115710509F46BC0FB012089318942899B
:1057D000538984859585A685B785281739074A0793
:1057E0005B0708F050C0F80184809580A680B780E0
:1057F0008085880E911CA11CB11CEBE1EE2EE2E02D
:10580000FE2EE00EF11EF70180819181A281B3810D
:1058100088159905AA05BB0571F080829182A28244
:10582000B382C8014B96AC01C501B4010E94B01D02
:10583000882309F074C0F80161857285E60FF71FAF
:10584000D38EF80184859585A685B7852089318911
:105850004289538982179307A407B50709F441C009
:105860002F5F3F4F4F4F5F4FF801208B318B428BA3
:10587000538BCB010196928781878050924090F4A0
:1058800080E090E050C0818592858050924008F47D
:10589000AACFCB010E944725892B09F0A4CF8FEF17
:1058A0009FEF41C0C8014B96AC01F7016081718147
:1058B000828193810E94091DC82F882381F5F801F8
:1058C0001286118680858F5F808790918E0689175A
:1058D000B8F2C8010E949521892B81F0F801C08798
:1058E000CFCF2F5F3F4F4F4F5F4F2487358746877E
:1058F00057872150304040405040B2CFC8010E94ED
:105900004725892B09F0BCCFF8018085815080871D
:1059100080E092E0928781878FEF9FEF04C00E9422
:10592000A7208FEF9FEFDF91CF911F910F91FF90F5
:10593000EF90DF90BF90AF909F908F9008952F923F
:105940003F925F926F927F928F929F92AF92BF929F
:10595000CF92DF92EF92FF920F931F93CF93DF933B
:10596000FC015A016B01380149011701EE24FF24A3
:105970008701A1E05A2E80918D068823A9F1211478
:10598000310491F1309781F1EF01E614F704080535
:10599000190538F5A114B104C104D104A1F05520B2
:1059A00091F0C1010E943D2B2FEF8F3F920709F12B
:1059B00089930894A108B108C108D108A114B104C1
:1059C000C104D10461F7552029F00894E11CF11CB1
:1059D000011D111DE614F7040805190510F45520E2
:1059E000C9F6C801B70107C060E070E080E090E050
:1059F00002C05524CFCFDF91CF911F910F91FF901F
:105A0000EF90DF90CF90BF90AF909F908F907F905E
:105A10006F905F903F902F9008952F923F925F92EA
:105A20006F927F928F929F92AF92BF92CF92DF92AE
:105A3000EF92FF920F931F93CF93DF93FC015A01D4
:105A40006B01380149011701EE24FF248701B1E001
:105A50005B2E80918D068823A9F12114310491F1E8
:105A6000309781F1EF01E614F7040805190538F5C0
:105A7000A114B104C104D104A1F0552091F0B101E9
:105A800088810E94CE2B8F5F9F4F09F12196089449
:105A9000A108B108C108D108A114B104C104D104FE
:105AA00061F7552029F00894E11CF11C011D111D1E
:105AB000E614F7040805190510F45520C9F6C801C5
:105AC000B70107C060E070E080E090E002C05524BC
:105AD000CFCFDF91CF911F910F91FF90EF90DF908B
:105AE000CF90BF90AF909F908F907F906F905F907E
:105AF0003F902F900895FF920F931F93CF93DF93C2
:105B0000EC018B01FF2420E030E080918D0688239A
:105B1000F1F0672BE1F02097D1F088818823A9F07C
:105B2000D901AC0FBD1FB8018C910E94CE2B9C01F6
:105B3000F394AF2DBB27FE01EA0FFB1F8081882362
:105B400021F08FEF2F3F380761F7C90102C080E0D5
:105B500090E0DF91CF911F910F91FF900895FC018C
:105B600080918D06882339F0452B29F0309719F064
:105B7000623071051CF080E090E008951082CF0142
:105B80000895EF92FF920F931F93CF937C01C0E093
:105B90000E943F1E8C019C0148E16C2FC7010E94AE
:105BA0003E24C82FC8010E94571E8C2F9927CF91E1
:105BB0001F910F91FF90EF900895FC0180899189CA
:105BC000A289B3890196A11DB11D2485358546851D
:105BD000578582179307A407B50718F480E090E073
:105BE000089581E090E00895CF93DF93FC01EB01ED
:105BF00090E0309721F1672B11F18485882319F407
:105C0000892F99271EC080819181A281B3818883C9
:105C10009983AA83BB8384819581A681B7818C8374
:105C20009D83AE83BF8380859185A285B385888758
:105C30009987AA87BB8781E08C87982FE1CF80E086
:105C400090E0DF91CF910895FC01009781F01082E0
:105C50001182128213821482158216821782108694
:105C6000118612861386148681E090E008950895C7
:105C70008091180499278130910519F1823091059E
:105C800084F0029719F01092180408958091A504E9
:105C90009091A6040E944D0F8823B9F31092180426
:105CA0000895892B81F78091C4039091C503816089
:105CB0009093C5038093C4038FE395E00E94242E44
:105CC000089588EE93E00E94440F9093A604809379
:105CD000A5048091C4039091C5038E7F9093C50362
:105CE0008093C4038091A7049091A8040196909397
:105CF000A8048093A7048091FB0399278370907078
:105D0000892B21F08091FA03843098F58FE395E098
:105D10000E94242E8091C6039091C703892BC1F065
:105D20008091F90380FF18C08091FA03843080F4D9
:105D30008091A7049091A80465E070E00E94EC2E89
:105D4000892B31F48AE090E09093E5038093E4039B
:105D500082E08093180408958091A7049091A8048C
:105D600065E070E00E94EC2E892BF1F684E690E06D
:105D7000EBCF6FE375E08CEE93E00E94F42DCACF79
:105D8000FC014150504030F001900616D1F7319798
:105D9000CF010895882799270895629FD001739FA6
:105DA000F001829FE00DF11D649FE00DF11D929FB7
:105DB000F00D839FF00D749FF00D659FF00D9927F6
:105DC000729FB00DE11DF91F639FB00DE11DF91F1A
:105DD000BD01CF0111240895AA1BBB1B51E107C0CF
:105DE000AA1FBB1FA617B70710F0A61BB70B881F6B
:105DF000991F5A95A9F780959095BC01CD010895FA
:105E0000A1E21A2EAA1BBB1BFD010DC0AA1FBB1FBE
:105E1000EE1FFF1FA217B307E407F50720F0A21B30
:105E2000B30BE40BF50B661F771F881F991F1A949D
:105E300069F760957095809590959B01AC01BD01C7
:105E4000CF01089597FB092E05260ED057FD04D0EB
:105E5000D7DF0AD0001C38F4509540953095219535
:105E60003F4F4F4F5F4F0895F6F79095809570958F
:0A5E700061957F4F8F4F9F4F0895FB
:105E7A007800416E616C6F675F4368302020202094
:105E8A002020416E616C6F675F43683120202020BB
:105E9A002020416E616C6F675F43683220202020AA
:105EAA002020416E616C6F675F4368332020202099
:105EBA002020416E616C6F675F4368342020202088
:105ECA002020416E616C6F675F4368352020202077
:105EDA002020416E616C6F675F4368362020202066
:105EEA002020416E616C6F675F4368372020202055
:105EFA0020205542617420202020202020202020AC
:105F0A00202053706565645F4E6F7274682020208C
:105F1A00202053706565645F4561737420202020DA
:105F2A00202053706565645F546F70202020202004
:105F3A0020204E756D4F66536174732020202020F7
:105F4A002020506F732E4C6F6E67697475646520DC
:105F5A002020506F732E4C6174697475646520201B
:105F6A002020506F732E416C74697475646520200B
:105F7A0020205A656C6C656E7A61686C202020203E
:105F8A002020506F7765724F6E202020202020201D
:105F9A002020446562756731382020202020202087
:105FAA002020446562756731392020202020202076
:105FBA00202044656275673230202020202020206E
:105FCA00202044656275673231202020202020205D
:105FDA00202044656275673232202020202020204C
:105FEA00202044656275673233202020202020203B
:105FFA00202044656275673234202020202020202A
:10600A002020446562756732352020202020202018
:10601A002020446562756732362020202020202007
:10602A0020204465627567323720202020202020F6
:10603A0020204465627567323820202020202020E5
:10604A0020204465627567323920202020202020D4
:10605A0020204465627567333020202020202020CC
:10606A0020204465627567333120202020202020BB
:10607A002020F4016401FFFFFF48656C6C6F205714
:10608A006F726C6400000000000000000000000055
:10609A0000000000000000000000000000000000F6
:1060AA0000000000000000000000000000000000E6
:1060BA0000000000000000000000000000000000D6
:1060CA0000000000000000000003000000001F00A4
:1060DA0000003B0000005A00000078000000970012
:1060EA000000B5000000D4000000F3000000110118
:1060FA000000300100004E0100006D0100000000A8
:10610A0000001F0000003C0000005B000000790056
:10611A00000098000000B6000000D5000000F4005E
:10612A00000012010000310100004F0100006E0161
:04613A000000010060
:00000001FF
